:10000000B7C01895189518951895189503C01895A8
:10001000189518950FB617EE12BF739580FF0BC099
:100020000894809B88944795783019F4112719BF5C
:1000300082600FBE1895713011F49198FACF7A3022
:1000400029F4919A112719BF8160F3CF40FD919A4D
:1000500040FF91984695EDCF81E012E013BF899A59
:10006000889808958827772712E019BF80FFFECF70
:100070000895809BFECF8099FECF1BED12BF12E04A
:1000800018BF19BF772781FFFECF8D7F08952FEF0F
:100090002A95F1F71A95D9F7089518E0331F10F44F
:1000A000C69A01C0C698C79A26E02A95F1F7C79864
:1000B00021E02A95F1F71A9589F7089518E030E0C4
:1000C000330FB5993160C79A26E02A95F1F7C798A2
:1000D00021E02A95F1F71A9599F7089500001FED90
:1000E00017BBC798063839F0073829F0C49A1FEFB4
:1000F000CEDFC49804C0C4981FEFC9DFC49A1FEFB5
:10010000C6DF3CEACADF33E5C8DF0032B8F00023BF
:10011000AAF0A0E2D3DF333599F030E0BEDFC79A12
:1001200026E02A95F1F7C79821E02A95F1F73CEAF5
:10013000B4DF33E5B2DFAA9569F702C030E0ADDF86
:10014000063821F0073811F030E0A7DF10E19FDF1B
:10015000089541E487DF46E585DF42E583DF40E23D
:1001600081DF49E47FDF43E57DDF40E57BDF089504
:100170001FED1DBF11271BBF1FEF12BBC49A18BB79
:1001800010E117BB69DF789474DF4B31E9F3443534
:1001900019F46FDF042F68C1433511F4DADFF4CFAF
:1001A000463529F442E35EDF40E35CDFEDCF4637BE
:1001B00029F441E357DF40E355DFE6CF4437D9F474
:1001C00042E150DF43E14EDF40E24CDF48E24ADFEC
:1001D00040E348DF48E346DF48E644DF48E442DFE7
:1001E00046E840DF47E83EDF42E43CDF41E43ADFF7
:1001F00040E038DFC9CF403719F443E533DFC4CFDF
:10020000483719F48D9A959A2FC1493719F48D9A68
:1002100095982AC10231B9F00331A9F0083399F059
:10022000083689F0083279F0003369F0003259F06D
:10023000063849F0073839F0023429F0013419F052
:10024000083409F00EC1403511F448DF0DC14334C4
:10025000C9F40FDF0638A9F0073899F038E41DDF3C
:10026000362F1BDF352F19DF342F17DF023421F033
:10027000013411F010E20BDF11E02227510F621F51
:10028000F3C0EFC04336C1F4F4DE063831F007386E
:1002900021F030E402DF362F03C0362F32D0326037
:1002A000FCDE352FFADE342FF8DE023421F0013483
:1002B00011F010E2ECDED8C0423559F5063831F0C5
:1002C000073821F038E2E9DE362F03C0362F19D087
:1002D0003160E3DE352FE1DEF1DE432FC3DE063889
:1002E00079F0073869F030E2D8DE362FD6DE352FC8
:1002F000D4DEE4DE432FB6DE11E02227510F621F69
